:100000000C942A000C9445000C9445000C94450077
:100010000C9445000C94E6010C9413020C943B02E2
:100020000C9445000C947A010C9445000C94450006
:100030000C9445000C9445000C945D030C94450011
:100040000C9445000C9445000C9445000C9445001C
:100050000C94450011241FBECFE5D4E0DEBFCDBF18
:1000600010E0A0E6B0E0ECE0FEE002C005900D92EA
:10007000A239B107D9F710E0A2E9B0E001C01D92A2
:10008000A93EB107E1F70C94AD000C940000CF93AA
:10009000DF93CDB7DEB7E7E3F0E08FE18083E4E301
:1000A000F0E08CEF8083E1E3F0E084E08083E2E342
:1000B000F0E088E38083DF91CF910895CF93DF93C1
:1000C000CDB7DEB721970FB6F894DEBF0FBECDBF18
:1000D000F89480E29EE49093E6008093E500198214
:1000E0002FC08981482F552789819927880F991F0B
:1000F000FC01E455FF4F808191819C0128513C4FC8
:10010000CA01880F991FFC01EB52FF4F31832083F6
:100110002091E5003091E60089819927880F991F89
:10012000FC01EB52FF4F80819181A901481B590BC3
:10013000CA019093E6008093E50089818F5F8983EF
:100140008981883070F2789421960FB6F894DEBFDA
:100150000FBECDBFDF91CF910895CF93DF93CDB781
:10016000DEB727970FB6F894DEBF0FBECDBF0E9453
:1001700047000E9458010E944F030E949E03109264
:10018000D3008AEF92E09093A7008093A60088E4C2
:1001900093E09093A9008093A800789480919600B2
:1001A0008823E1F3109296000E9431060E94860493
:1001B00000C080919800813041F4109298008091A5
:1001C000D300882311F40E945E0080919600813054
:1001D00081F7109296001A821CC080E690E00E947F
:1001E000D8038A8199270E94220487E690E00E9422
:1001F000D8038A819927880F991FFC01EB52FF4F82
:10020000808191810E9422040E9413048A818F5F61
:100210008A838A81893008F38091D4008595992753
:1002200087FD909590939A00809399002091990072
:1002300030919A00CE0103964AE050E0BC01C9011A
:100240000E94C106CE010396DC01FD010190002051
:10025000E9F73197CF018A1B9B0B89836AE080E025
:100260000E940D068AE690E00E94AF059DE089811C
:10027000292F281B822F682F80E00E940D06CE01B7
:1002800003960E94AF0595CFCF93DF93CDB7DEB72E
:10029000F894E9E5F0E089E180837894DF91CF91EB
:1002A0000895CF93DF93CDB7DEB7DF91CF91089557
:1002B000CF93DF93CDB7DEB7E3E5F0E082E0808354
:1002C000EFE4F0E01082EEE4F0E082E08083EAE424
:1002D000F0E084EF91E091838083E8E4F0E080ED4A
:1002E00097E091838083E9E5F0E089E18083DF9105
:1002F000CF9108951F920F920FB60F9211242F9352
:100300003F934F935F936F937F938F939F93AF939D
:10031000BF93EF93FF93CF93DF93CDB7DEB70E94E8
:1003200078068091D2008F5F8093D2008091D200B6
:100330008834C9F581E0809397001092D2008091B3
:100340009D008F5F80939D0080919D00853029F4F2
:1003500010929D0081E08093980080919B008F5FB8
:1003600080939B0080919B00843641F410929B0007
:1003700081E08093940081E08093960080919B00BF
:10038000823319F481E08093960080919C008F5F06
:1003900080939C0080919C008A3029F410929C00EC
:1003A00081E080939500DF91CF91FF91EF91BF9114
:1003B000AF919F918F917F916F915F914F913F91FD
:1003C0002F910F900FBE0F901F9018951F920F92B4
:1003D0000FB60F9211242F933F934F935F936F9318
:1003E0007F938F939F93AF93BF93EF93FF93CF939D
:1003F000DF93CDB7DEB7E091A600F091A700099595
:10040000DF91CF91FF91EF91BF91AF919F918F912C
:100410007F916F915F914F913F912F910F900FBE00
:100420000F901F9018951F920F920FB60F921124E4
:100430008F93AF93BF93EF93FF93CF93DF93CDB79A
:10044000DEB7A2E3B0E0E2E3F0E080818B7F8C9343
:10045000A8E3B0E0E8E3F0E080818F7E8C93DF9149
:10046000CF91FF91EF91BF91AF918F910F900FBE00
:100470000F901F9018951F920F920FB60F92112494
:100480002F933F938F939F93AF93BF93EF93FF93DC
:10049000CF93DF93CDB7DEB72297DEBFCDBFA2E308
:1004A000B0E0E2E3F0E0808184608C93ECE4F0E083
:1004B00011821082A8E4B0E0809192009927880F01
:1004C000991FFC01EB52FF4F8081918111969C9303
:1004D0008E9380919200882339F4A8E3B0E0E8E39A
:1004E000F0E0808180618C9380919200282F3327E7
:1004F0003A83298389819A8182309105C1F12981CA
:100500003A812330310554F489819A81009789F02A
:1005100029813A8121303105D9F04EC089819A81F3
:100520008330910599F129813A8124303105E9F12F
:1005300043C0A8E3B0E0E8E3F0E0808180618C9301
:10054000A8E3B0E0E8E3F0E0808181608C9334C000
:10055000A8E3B0E0E8E3F0E080818E7F8C93A8E32D
:10056000B0E0E8E3F0E0808182608C9325C0A8E3EE
:10057000B0E0E8E3F0E080818D7F8C93A8E3B0E009
:10058000E8E3F0E0808184608C9316C0A8E3B0E0DB
:10059000E8E3F0E080818B7F8C93A8E3B0E0E8E3B0
:1005A000F0E0808188608C9307C0A8E3B0E0E8E3C6
:1005B000F0E08081877F8C93809192008F5F8093A1
:1005C000920080919200893010F010929200229651
:1005D000F894DEBFCDBFDF91CF91FF91EF91BF9136
:1005E000AF919F918F913F912F910F900FBE0F90E0
:1005F0001F901895CF93DF93CDB7DEB780919E0003
:1006000090919F000097B1F4E6E4F0E08081918141
:100610009093A5008093A400AEE4B0E0EEE4F0E097
:1006200080818F7B8C9381E090E090939F008093FA
:100630009E002BC0E6E4F0E0808191819093A300BE
:100640008093A200AEE4B0E0EEE4F0E0808180644C
:100650008C932091A2003091A3008091A4009091EE
:10066000A500A901481B590BCA019093A1008093D2
:10067000A00010929F0010929E008091A000909187
:10068000A1009093E8008093E700DF91CF91089557
:10069000CF93DF93CDB7DEB7DF91CF910895CF939E
:1006A000DF93CDB7DEB7E7E2F0E01082E6E2F0E0FC
:1006B0008FEE8083DF91CF9108951F920F920FB636
:1006C0000F9211242F933F938F939F93EF93FF9358
:1006D000CF93DF93CDB7DEB7E6E2F0E010828091F2
:1006E00093009927E4E2F0E020813181880F991F7F
:1006F000FC01E455FF4F31832083809193008F5F8D
:100700008093930080919300883010F010929300B2
:10071000E7E2F0E0809193008083E6E2F0E08FEE84
:100720008083DF91CF91FF91EF919F918F913F91C6
:100730002F910F900FBE0F901F901895CF93DF93BE
:10074000CDB7DEB7E9E2F0E080E18083E0E4F0E0FD
:100750001082EAE2F0E088E18083E0E4F0E086E8FD
:100760008083EBE2F0E082EC8083DF91CF9108950B
:10077000CF93DF93CDB7DEB721970FB6F894DEBFE6
:100780000FBECDBF8983EBE2F0E0808199278072B4
:1007900090700097C1F3ECE2F0E0898180832196AC
:1007A0000FB6F894DEBF0FBECDBFDF91CF91089595
:1007B000CF93DF93CDB7DEB726970FB6F894DEBFA1
:1007C0000FBECDBF9E838D838D819E81DC01FD0197
:1007D00001900020E9F73197CF018A1B9B0B9C8386
:1007E0008B831A8219820FC029813A818D819E8163
:1007F000F901E80FF91F80810E94B80389819A816D
:1008000001969A83898329813A818B819C81821701
:10081000930750F726960FB6F894DEBF0FBECDBFF4
:10082000DF91CF910895CF93DF93CDB7DEB780915D
:100830006E000E94B80380916F000E94B803DF91A0
:10084000CF910895CF93DF93CDB7DEB766970FB6FC
:10085000F894DEBF0FBECDBF9E8B8D8B8D899E8998
:100860004AE050E09E012F5F3F4FB9010E94C10650
:10087000CE0101960E94D80366960FB6F894DEBFAB
:100880000FBECDBFDF91CF910895CF93DF93CDB74A
:10089000DEB722970FB6F894DEBF0FBECDBF8A83B6
:1008A00087E089831FC08A81482F55278981282F97
:1008B000332727FD309581E090E0022E02C0880F9B
:1008C000991F0A94E2F7842395231816190624F435
:1008D00081E30E94B80303C080E30E94B8038981CA
:1008E0008150898389818823F4F680916E000E946B
:1008F000B80380916F000E94B80322960FB6F89457
:10090000DEBF0FBECDBFDF91CF910895CF93DF93B0
:10091000CDB7DEB70E94A90463E080E00E940D0617
:1009200080E790E00E94AF0562E081E00E940D0642
:100930008BE790E00E94AF05E0E3F0E0808199272B
:10094000807290700097C1F70E94A904DF91CF9147
:100950000895CF93DF93CDB7DEB781E00E94E40521
:10096000DF91CF910895CF93DF93CDB7DEB7269770
:100970000FB6F894DEBF0FBECDBF9E838D838AE095
:1009800090E09C838B831CC082E390E09A838983F0
:100990000EC08D819E8101979E838D838D819E8166
:1009A0000097B9F789819A8101979A838983898110
:1009B0009A81009799F78B819C8101979C838B8307
:1009C0008B819C81009701F726960FB6F894DEBFC5
:1009D0000FBECDBFDF91CF910895CF93DF93CDB7F9
:1009E000DEB721970FB6F894DEBF0FBECDBF898367
:1009F0008981992781709070882341F0A5E3B0E048
:100A0000E5E3F0E0808180618C9307C0A5E3B0E06E
:100A1000E5E3F0E080818F7E8C9389819927827055
:100A20009070009741F0A5E3B0E0E5E3F0E080814D
:100A300080628C9307C0A5E3B0E0E5E3F0E080813D
:100A40008F7D8C938981992784709070009741F0F5
:100A5000A5E3B0E0E5E3F0E0808180648C9307C01B
:100A6000A5E3B0E0E5E3F0E080818F7B8C938981A2
:100A7000992788709070009741F0A5E3B0E0E5E316
:100A8000F0E0808180688C9308C0A5E3B0E0E5E3E6
:100A9000F0E090818FE789238C9321960FB6F8942C
:100AA000DEBF0FBECDBFDF91CF910895CF93DF930F
:100AB000CDB7DEB7A5E3B0E0E5E3F0E08081846088
:100AC0008C9381E090E00E94B304A5E3B0E0E5E3FD
:100AD000F0E080818B7F8C93DF91CF910895CF934D
:100AE000DF93CDB7DEB722970FB6F894DEBF0FBE07
:100AF000CDBF8A838A8182958F70898389810E9484
:100B0000ED040E9456058A810E94ED040E9456055C
:100B100022960FB6F894DEBF0FBECDBFDF91CF9106
:100B20000895CF93DF93CDB7DEB721970FB6F89432
:100B3000DEBF0FBECDBF8983A5E3B0E0E5E3F0E003
:100B4000808188608C9389810E946F0521960FB601
:100B5000F894DEBF0FBECDBFDF91CF910895CF9344
:100B6000DF93CDB7DEB724970FB6F894DEBF0FBE84
:100B7000CDBF9C838B838B819C81DC01FD01019027
:100B80000020E9F73197CF018A1B9B0B8A831982DA
:100B90000EC0898199279C018B819C81F901E80F06
:100BA000F91F80810E94910589818F5F89839981D6
:100BB0008A81981770F324960FB6F894DEBF0FBEA3
:100BC000CDBFDF91CF910895CF93DF93CDB7DEB73F
:100BD00021970FB6F894DEBF0FBECDBF898381E0A9
:100BE00090E00E94B304A5E3B0E0E5E3F0E080818B
:100BF000877F8C9389810E946F05A5E3B0E0E5E3D0
:100C0000F0E0808188608C9321960FB6F894DEBF67
:100C10000FBECDBFDF91CF910895CF93DF93CDB7B6
:100C2000DEB723970FB6F894DEBF0FBECDBF8A8321
:100C30006B838A81882319F48B81805889838A8108
:100C4000813019F48B818054898389810E94E40565
:100C500023960FB6F894DEBF0FBECDBFDF91CF91C4
:100C60000895CF93DF93CDB7DEB781E090E00E9487
:100C7000B304A5E3B0E0E5E3F0E08081877F8C93E7
:100C800083E00E94ED040E94560585E090E00E94FA
:100C9000B30483E00E94ED040E94560581E090E0D9
:100CA0000E94B30483E00E94ED040E94560582E096
:100CB0000E94ED040E94560581E090E00E94B3047A
:100CC00088E20E94E4058EE00E94E40581E00E9433
:100CD000E40588E890E00E94AF056AE081E00E94A8
:100CE0000D068DE890E00E94AF05DF91CF91089549
:100CF000CF93DF93CDB7DEB721970FB6F894DEBF61
:100D00000FBECDBF1982E0E3F0E0808199278071AA
:100D10009070009711F081E08983E0E3F0E080813A
:100D2000992788709070009721F0898193E0892736
:100D30008983998180916900292F281B822F8983BB
:100D40008981992787FD909581709070882381F023
:100D500080916900982F8981890F8093690089812A
:100D6000982F92708091D400890F81508093D40085
:100D700021960FB6F894DEBF0FBECDBFDF91CF91A5
:100D80000895FB019F01E8944230C4F04532B4F469
:100D90004A3029F497FB1EF4909581959F4F642F5C
:100DA00077270E94F206805D8A330CF0895D81937B
:100DB000CB010097A1F716F45DE251931082C901AF
:100DC0000C94E206DC01FC0101900020E9F7329767
:100DD000AE17BF0730F47C916081708331976D93BB
:100DE000F7CF0895AA1BBB1B51E107C0AA1FBB1F69
:100DF000A617B70710F0A61BB70B881F991F5A95A7
:0C0E0000A9F780959095BC01CD010895E4
:100E0C004B2000000000003D0001202020000D0AB6
:100E1C004550492D5465737465720056657273693B
:100E2C006F6E20302E3263006875687500416B6BF5
:020E3C0075003F
:00000001FF
